:020000040000FA
:06000000D38CD38A25D148
:08000800F2B407D0A498110026
:04001000F7D7F6D751
:0800180025D0F2941C500BE00E
:10002000E84C10D0E84C17D08B8E67C0D7FF66C065
:10003000D6FF1C0611001C2A67C0D7FF948E66C02D
:10004000D6FF11001D9E82BE1D8E1C2A69C0D7FFDF
:1000500068C0D6FF1100948E1B80D59E1C6A1100CB
:10006000110012009E9CE8CF05F1D8CF06F1E0CF39
:1000700007F1F6CF0AF1F7CF0BF1F5CF0DF1F4CF81
:100080000EF1F3CF0FF101011EA808D06E51425FAF
:100090006F51435B7051445B08E309D06E514227B6
:1000A0006F5143237051442302E31E8EA191344EBD
:1000B00002900201133F04D0143F02D0143F00D03D
:1000C000C1A40ED0C290322A030EC11407E0C3505F
:1000D000C11404E0C350C11401E0C350C28073D006
:1000E000560EE81C9916C4500427C3500327D8B0F5
:1000F000042BC4500627C3500527D8B0062BC45084
:100100000827C3500727D8B0082BC4500A27C3506C
:100110000927D8B00A2B012F56D0400E016F03C219
:1001200036F204C237F205C238F206C239F207C20B
:100130003AF208C23BF209C23CF20AC23DF2036B3A
:10014000046B056B066B076B086B096B0A6B3180E0
:10015000318239D0E81C9916C4500C27C3500B27A4
:10016000D8B00C2BC4500E27C3500D27D8B00E2B7F
:10017000C4501027C3500F27D8B0102BC4501227DB
:10018000C3501127D8B0122B022F1DD0400E026F82
:100190000BC23EF20CC23FF20DC240F20EC241F25F
:1001A0000FC242F210C243F211C244F212C245F22F
:1001B0000B6B0C6B0D6B0E6B0F6B106B116B126B73
:1001C0003180318400D00101292AA22F09D0190ED3
:1001D000A26F2A2A0084008C04668B7C04660406C5
:1001E000A32F07D0F50EA36F2B2A00840088008A66
:1001F0001E82A42F10D0A52F0ED008BC05D0890ECA
:10020000A46F0A0EA56F05D0089C900EA46F0A0E6D
:10021000A56F2C2A0080234E1E8A8CEC04F09EAC25
:1002200003D09E9C222A2FD70AC1F6FF0BC1F7FFED
:100230000DC1F5FF0EC1F4FF0FC1F3FF07C1E0FFD1
:0E02400005C1E8FF06C1D8FF1000A498100009
:02024E000000AE
:10025000D0CF60F00400D388899092906F6A8A684A
:10026000000E936E1F9AD08ED098D082D08000015D
:10027000000E936E000E946EFC6A22EEFFF00001F9
:10028000730ED36E939C8A8C939E8A9EF86A616BE0
:10029000626B636B646B090E656FF29EF29C0101E9
:1002A00003EC0EF0949C046AD0A604060101949A13
:1002B000949892988B9A8B988998076A096A086A29
:1002C0000A6A076A176A196A1A6A0886050E1B6F96
:1002D0000001D56AD580D59CF294F28AD59ED76A62
:1002E000D66AF1841B6A1C6A1C2A9A6B9B6B776B1B
:1002F000766B762B762B916B1B80756B0101786A80
:100300001F0E796E766A1F0E776E746A1F0E756EF9
:100310000F0E7A6E140E496FFF0E7B6E000E486F43
:100320007F6A7F827E6A7E8E6F6A6B686A6A6F6A96
:100330006F8C899092806E6A6D6A6B686A6A6C6A6B
:10034000226A0101206A20721F6A1E6A8E6B8D6B01
:10035000746B756B796B0D0E7A6F080E7B6F0A0EDE
:100360007C6F776B1E96DEEC03F0A588A498A398AB
:10037000D0B603D01F86010E8D6F0101256A266A53
:10038000276A286A2D6A190EA26FF50EA36F890ECF
:10039000A46F0A0EA56F91689068886A876AB76A29
:1003A000B78CB7800201C26AC280C288C28AC28486
:1003B000C16AC188C06AC082E86AE886E888E88ABB
:1003C000C012C08E9A6A9A8E0F0EB86E926EB8984E
:1003D000996AC2809F9C9E9C9D8CC282200E016F58
:1003E000400E026F326A036B046B056B066B076B82
:1003F000086B096B0A6B0B6B0C6B0D6B0E6B0F6B49
:10040000106B116BF28EF28CD180016A026A06D0F9
:10041000014E029402B009D0025007E11E0E346E64
:10042000020E016E028002840400000108B094EC08
:100430000DF009A815EC06F000B2F3EC08F000B4DA
:10044000EFEC08F000B617EC09F01BB07CEC0AF0FA
:100450001EA204D001011E9297EC02F01EAA2CD01D
:1004600001011E9A585115E11EA010D01E9018A827
:100470001F8218A21F9418A81F8218A81F8418B6DC
:1004800005D0765102E11E7801D01F8888EC03F078
:1004900012D0E82C0ED01EA009D01E9018A61F82E4
:1004A00018A61F9418A81F8218A81F84C4EC0EF069
:1004B00002D0C4EC0EF08F6F1EAE03D0010107EC2A
:1004C00004F000AC04D0009C010135EC0EF000AA51
:1004D00004D0009A010136EC0EF000A004D0010116
:1004E000009037EC0EF031B0A5EC0BF008EF02F005
:1004F000D890E846E846E890FD26000EFE2212005D
:10050000F29EF29CE8CF61F0FDCF62F0FECF63F087
:10051000FFCF64F0FC6A7F0E04260001652F02EF16
:0805200002F0FF003D0C150C78
:08052800210E80EC02F0765177
:10053000030D82514EE0E84C51D0E84C54D0E84CC9
:1005400057D082C1F6FFF76AF636F736F690F86AAA
:100550007B0EF626310EF722000EF8220900F55028
:100560007603F3CF83F1F4CF84F1856B0900F55066
:100570007603F3508427F4508523F29C83C16EF1F7
:1005800084C16FF185C170F1F28C87517603F3CF8E
:1005900085F1F4CF86F1F334856FF434866F07E28A
:1005A00088518803F3508527F450862302E3856938
:1005B000866985390F0B836F8639F00B8313863973
:1005C0000F0B846FF29C83C172F184C173F1F28CC2
:1005D00012007B0EF326330EF4220ED07B0EF32690
:1005E000360EF42209D07B0EF326390EF42204D005
:1005F0007B0EF3263C0EF422F3CFF6FFF4CFF7FF89
:10060000F86A0900F5CF83F10900F5CF84F10900FC
:10061000F5CF85F1B2D7899092906F6A8A68000E03
:10062000936E1F9ADEEC03F01E961E981F901F9883
:100630001F9A2CC095F18E2B010C1F921F988D5183
:1006400006E095512C5C1408D8B0D10C06D01E9849
:1006500095512C5C0208D8B0D20C8E2B020C3BC2F8
:10066000E8FF0208D8A0030C3DC2E8FF8C5DD8B0BB
:10067000040C2CC095F18E2B050C95512C5C0708B1
:10068000D8B0D30C8E2B060C208020821FB609D048
:100690001E9891BF1E88915104E09145E880786FC3
:1006A0000AD01FA2070C78C180F108801FA403D0D4
:1006B000800E786F1F966B686A6A6F6A6F8C89907C
:1006C00092801F921E861E8C010E766F6A6AC00E83
:1006D0006B168E2B2CC095F1080C95512C5C0208E2
:1006E000D8B0D40C8E2B090C39C2E8FFB208D8A0C0
:1006F000100C3F0E6B121F928D6B8E2B110C1FA2D4
:1007000021D01FB616D01F861F9280C178F11AD053
:1007100092C123F08E517AEC02F07DD78ED79FD70D
:10072000ACD7B2D7DAD7E0D7EAD71F96800E786F6A
:1007300009D01F9278C180F108801FB4F6D71E96A9
:100740001F98776B1F8A1FB81E961EA606D078C109
:1007500077F108A67FC177F101D0776B7651776387
:1007600044D0D8A43DD01FB035D01FB833D01EBC64
:1007700025D01EB6120C1F9A899092906F6A8A68D3
:10078000000E936E1F9A2CC095F18D6B010E8E6F2B
:10079000130CE84AE868E8CF8DF1E86AE8CF8EF1FB
:1007A000899092906F6A8A68000E936E1F9A1F86D6
:1007B0001E961F901F981F9AA00E04268990929053
:1007C0006F6A8A68000E936E1F9A1E9C6A6AC00E3A
:1007D0006B16200C1E781F9878C177F11E86210CAD
:1007E0001FA0220C1E96776B230C7651D8A405D03F
:1007F0001EBC03D01E8C3F0E6B12776503D0764B68
:100800007669240C7607D8A0766B250C150CA1B15F
:100810003BD0744B752BA18196C19CF197C19DF182
:1008200098C19EF199519C5F9A519D5B9B519E5B33
:1008300096C199F197C19AF198C19BF1020116C234
:100840001CF217C21DF218C21EF219C21FF21AC200
:1008500020F21BC221F226C22CF227C22DF228C29E
:100860002EF229C22FF22AC230F22BC231F2166BBD
:10087000176B186B196B1A6B1B6B26692769286934
:1008800029692A692B6912001200208093EC02F07A
:100890005D6F4F515D5D1EE34F51060DF3CFF6FFC7
:1008A000F4CFF7FFD50EF626280EF722F86AA68EAB
:1008B0000900F5CF7BFF0900F5CF7AFF0900F5CFDE
:1008C0004AF10900F5CF4BF10900F5CF48F10900D5
:1008D000F5CF49F1120020825151030B060DF3CFE1
:1008E000F6FFF4CFF7FF530EF626290EF722F86A2B
:1008F000A68E0900F5CF52F10900F5CF53F109009A
:10090000F5CF54F10900F5CF55F10900F5CF56F1B7
:100910000900F5CF57F112000101A68E20A0B5DF26
:1009200020A2D9DF43390F0BF66E4439F00BF612D3
:1009300044390F0BF76EF690F7B605D06B0EF6261E
:10094000290EF72209D0F796F6506B08F66EF7508D
:10095000D8A0E83C3108F76E0900F550636F7203C8
:10096000F3CF5CF1F4CF5DF10900F5507303F3CFE1
:100970005EF1F4CF5FF17203F3505D27F4505E2314
:1009800063517303F3505D27F4505E23F5AE04D03A
:1009900072515E5F73515F5B010E5C277F0E5D23BA
:1009A0007F0E5E23990E5D5F190E5E5B32E3CC0E07
:1009B0005D5DCC0E5E590FE25D514903F4CF60F1ED
:1009C0005E5149036051F326E86AF422F3CF79FFC0
:1009D000F4CF78FF20D059510DE04BC15CF14A5D56
:1009E000D8A05C07D8806D54D8A05C07796E5CC134
:1009F00078FF11D04AC179FF4BC178FF0CD05C6BF6
:100A0000595107E06D24D8B05C2B796E5CC178FF3A
:100A100002D0796A786A5251422553514321466F78
:100A200054514421476F46390F0BF66E4739F00B8E
:100A3000F61247390F0BF76EF690F7B605D06B0E2E
:100A4000F626290EF72209D0F796F6506B08F66EB7
:100A5000F750D8A0E83C3108F76E0900F550636FF5
:100A60007203F3CF5CF1F4CF5DF10900F55073032D
:100A7000F3CF5EF1F4CF5FF17203F3505D27F450D2
:100A80005E2363517303F3505D27F4505E23F5AE8C
:100A900004D072515E5F73515F5B010E5C277F0E65
:100AA0005D237F0E5E23990E5D5F190E5E5B32E360
:100AB000CC0E5D5DCC0E5E590FE25D514903F4CF63
:100AC00060F15E5149036051F326E86AF422F3CFE6
:100AD00077FFF4CF76FF20D059510DE04BC15CF188
:100AE0004A5DD8A05C07D8806D54D8A05C07776EAB
:100AF0005CC176FF11D04AC177FF4BC176FF0CD0A5
:100B00005C6B595107E06D24D8B05C2B776E5CC1EB
:100B100076FF02D0776A766A5551422556514321B5
:100B2000466F57514421476F46390F0BF66E4739D0
:100B3000F00BF61247390F0BF76EF690F7B605D0AB
:100B40006B0EF626290EF72209D0F796F6506B08A1
:100B5000F66EF750D8A0E83C3108F76E0900F55062
:100B6000636F7203F3CF5CF1F4CF5DF10900F550D0
:100B70007303F3CF5EF1F4CF5FF17203F3505D279F
:100B8000F4505E2363517303F3505D27F4505E23EA
:100B9000F5AE04D072515E5F73515F5B010E5C274E
:100BA0007F0E5D237F0E5E23990E5D5F190E5E5BE7
:100BB00032E3CC0E5D5DCC0E5E590FE25D51490310
:100BC000F4CF60F15E5149036051F326E86AF422E4
:100BD000F3CF75FFF4CF74FF20D059510DE04BC116
:100BE0005CF14A5DD8A05C07D8806D54D8A05C0742
:100BF000756E5CC174FF11D04AC175FF4BC174FFA3
:100C00000CD05C6B595107E06D24D8B05C2B756E2D
:100C10005CC174FF02D0756A746A21500000E82C30
:040C2000FDD71200EA
:0C0C2400190E80EC02F00101A68E09B050
:100C30000AD009B23ED009B431D009B624D02AC0B6
:100C400026F1098612000ABE43D00AA005D00EC0C4
:100C50000CF00A8E0A903CD00AA205D00FC00CF00E
:100C60000A8E0A9235D00AA405D010C00CF00A8E64
:100C70000A942ED00AA605D011C00CF00A8E0A964E
:100C800027D00988120026512A5C3408D8B0F10C0C
:100C900009848B9A280EA0EC06F0120026512A5CDB
:100CA0003E08D8B0F20C09828B9A280EA0EC06F010
:100CB000120026512A5C3F08D8B0F30C09808B9AA9
:100CC000280EA0EC06F00C6A0D6A0B6A099A0A8ECF
:100CD00009BA84D0098A500EF66E230EF76EA68EDE
:100CE000F86A92EC02F0206F0C50205D5DE20A9EE3
:100CF000099C099A099E1F6B1200F55019E0A8087B
:100D000002E1A20E1DD0F550B80802E1B50E18D0D0
:100D1000F550BF080BE2230EF76EF86AC00EF55CC3
:100D2000100FF66ED8B0F72AA68E0800F55008D03E
:100D300008A8DDD7089819C117F11AC118F11200D7
:100D400001018B982F6F306F2F3BF00E94162F13ED
:100D500030138B500F092F158B6E898824D88998F2
:100D600022D80F0930158B6E898889980F0E94123E
:100D7000120000B4D7D98B9A0F0E94128B888988F1
:100D800012D882A607D0D890314B322BD8B0096A3E
:100D9000060002D0316B326B899805D8898803D858
:100DA00089988B98120012000CC020F1216BD8900A
:100DB000203721372051F6262151F722A68E09002F
:100DC000F5CF20F10900F5CFF7FF20C1F6FF0900AC
:100DD000F6CF17F1F7CF18F1F5CF0BF009BC07D01C
:100DE000C8DF098C0B50E88E8B9AA0EC06F008B493
:100DF00055D1BFDF8B8A0D5004E1FF0E0C1401E1C9
:100E00008B9A09BE5CD182D98BAA77D70F0EF56475
:100E100074D7200EF56071D70101100E72D0020E4A
:100E20005BD901EE27F015C020F1F6D848D1010EAC
:100E30001F6F3A0E1E6F098E69D9F5CFE9FF07B40F
:100E4000F5CF15F163D9F5CFEAFF07B4F5CF16F169
:100E50000794EECF15F0270E1C6F010E1D6F01EEEB
:100E600027F015C020F12051DCD807941CC1E9FF00
:100E70001DC1EAFF1F4F099EEE50E9CF1CF1EACFDA
:100E80001DF15ED7040E28D901EE27F016C020F11F
:100E9000C3D815C020F1C0D812D1020E1DD9166AD0
:100EA000C6D801EE27F021C120F1B6D808D1050E31
:100EB00013D9BDD801EE27F023C120F1ADD822C14E
:100EC00020F1AAD821C120F1A7D81C4B1D2BF7D0A7
:100ED000040E02D9166A15AE04D0099E151E152AF5
:100EE000159EA5D801EE27F022C120F195D821C189
:100EF00020F192D8200E276F2D0E09AE276F098E94
:100F0000DED0F55C7AEC02F08AD7BCD7C6D7CFD753
:100F1000DFD742D05ED063D08AD707D06DD087D7D5
:100F200086D785D784D783D782D7060ED5D816AE75
:100F300006D0099E151E161E154A162A169E226BED
:100F4000236B15500A0DF3CF20F1F4CF21F1165089
:100F50000A0DF3502127F4502223040E236FD8905A
:100F6000223321332033232FFAD720C115F021C19A
:100F700016F05DD801EE27F0200EEE6E22C120F1B2
:100F80004BD821394ED82E0EEE6E21514AD82D0E57
:100F900009AE276F098E93D0060E9ED816AE06D0E6
:100FA000099E151E161E153E162A169E40D801EEE5
:100FB00027F023C120F130D822C120F12DD821C142
:100FC00020F12AD8200E276F2D0E09AE276F098E2B
:100FD00076D09CD8099EF550E88E8B9AB1D60784BE
:100FE000078694D8F5CF39F191D8F5CF3AF1079823
:100FF00039513A6507881200088888D8F5CFE9FF8B
:1010000085D8F5CFEAFFEF500C6E0D6A17C119F1C4
:1010100018C11AF179EF06F0203903D8205101D810
:1010200012000F0B300F1E65070FEE6E1200F29EBE
:10103000FDCF11F1FECF12F1FFCF13F10600F28EBA
:101040000884D8900F0E256F010E206F216B226B44
:10105000236B15361636213722372337204F1200DF
:1010600001EE20F0EC5007E0030FE8B6EF6EEF5012
:10107000300FE8BEEF6EEC5007E0030FE8B6EF6EFE
:10108000EF50300FE8BEEF6EEC50E3E0030FE8B630
:10109000EF6EEF50300FE8BEEF6EDBD7010E206F22
:1010A000252FDED7089405000101F29E1151FD6E37
:1010B0001251FE6E1351FF6EF28E0101D1D70794CB
:1010C0001CC1E9FF1DC1EAFF1F4F099EEE50E9CF89
:1010D0001CF1EACF1DF134D61F6F18D8F5CFE9FF08
:1010E00007B4F5CF15F112D8F5CFEAFF07B4F5CF65
:1010F00016F10794EECF15F0EECF16F0098E3A0EEA
:101100001E6F270E1C6F010E1D6F1200A68E17C1D9
:10111000F6FF18C1F7FFF86A0900F6CF17F1F7CF0D
:1011200018F11200009489988B888B9A0F0E9412F4
:1011300082A4189E82B4188E82A0189C82B0188C4B
:10114000008600A81200009882A6179E82B6178E0D
:1011500082A4179C82B4178C82A2179A82B2178A33
:1011600082A0179882B0178882A6189882B618882D
:1011700082A2189A82B2188A8B8A8B9882A61796B6
:1011800082B6178682A4179482B4178482A217921B
:1011900082B2178282A0179082B0178082A618961A
:1011A00082B6188682A4189482B4188482A21892F7
:1011B00082B2188282A0189082B0188018503F0B1B
:1011C000346303D03BC138F11200382F12003BC109
:1011D00038F100821E8018503F0B346F120001015D
:1011E00009A812009FD70101009201011850200B9D
:1011F000376301D01AD01F0E0426376F08B615D0FA
:1012000018BA13D007B00BD007A60FD00780030E73
:10121000195CD8B41F800101040E1B6F06D0079023
:101220001F900101050E1B6F0880120012000101C2
:1012300000961850C00BE8BEE87C356301D0120060
:10124000356115D036077F0E366154D0040E042662
:1012500008A61A6A800E366F08B62AD007B01BD0CF
:1012600007961906D8B041D01A0E196E3ED0362B0B
:10127000810E36653FD0080E042608A61A6A800E35
:10128000366F08B61BD007B01FD00796192A1B0E61
:101290001960196A2AD0E9CF08F1EACF09F115C11E
:1012A000E9FF16C1EAFF395107A8EF62EF0618D02F
:1012B0000101000E7863780701011CD00101FF0EC7
:1012C0007863782B010116D0E9CF08F1EACF09F154
:1012D00015C1E9FF16C1EAFF3A5107A8EF62EF2AEC
:1012E00008C1E9FF09C1EAFF00D01950150F106EBF
:1012F00009980A841850C00BE8BEE87C356F1200CC
:021300001200D9
:0E130200150E80EC02F017C093F09369939FD4
:1013100008B60CD00F0E196209D007A007D0936948
:10132000939F2BC077F0010E756F000C76517527D7
:10133000000C77512B5C0508D8B0E10C906B00EEE7
:1013400086F0E9CF3EF1EACF3FF1080E746F330E1D
:101350006A6F030E796F220E7A6F230E786F6FD14A
:10136000756B000C0A0E7B6F550E6B6FC7D900EEC4
:101370007CF0E9CF40F1EACF41F19BD13EC1E9FFDA
:101380003FC1EAFF1DC0EEFFE9CF3EF1EACF3FF1DA
:10139000742F2ED1756B000C77512B5C0508D8B0DB
:1013A000E10C330E6A6F000E796F220E7A6F230EF6
:1013B000786F45D1756B000C330E6A6F000E796F34
:1013C000220E7A6F2CD1756B290E756F1D6ACC0EAB
:1013D0006A6F290E7A6F230E786F31D1756B000C0E
:1013E0001DC071F01DAE03D093BF09D00ED01B9469
:1013F000756B1B80A50E876F5A0E866F000C752BC0
:1014000075C07AF0BE0E6A6F0AD11BB60DD01B866E
:10141000906B070E796F090E746F00EE86F0E9CFBE
:101420003EF1EACF3FF1E4D03EC1E9FF3FC1EAFF20
:101430001DC0EEFFE9CF3EF1EACF3FF1742FD8D0C7
:10144000756B1B941B921B801B961B88000C000C59
:10145000752B54D9080E746F00EE86F0EECF6AF04B
:10146000E9CF3EF1EACF3FF175C07AF0D8D03EC166
:10147000E9FF3FC1EAFFEECF6AF0E9CF3EF1EACFE4
:101480003FF1742FCCD0752B75C079F0220E7A6F96
:10149000BE0E6A6F090E746F906B00EE86F0E9CF96
:1014A0003EF1EACF3FF1BBD03EC1E9FF3FC1EAFFC9
:1014B0001DC0EEFFE9CF3EF1EACF3FF1742F98D087
:1014C00040C1E9FF41C1EAFF905106E186C0EEFF4D
:1014D00087C0EEFF8A7E02D0EE50EE50E9CF40F199
:1014E000EACF41F1734F5BD01D6A550E6A6F0A0E49
:1014F0007A6F230E786FA3D01B9A00012D0E6E6FAA
:1015000075516E65000C7AEC02F0FED612D72AD720
:1015100035D742D751D764D778D726D026D098D799
:10152000A6D7C2D756D022D022D022D022D022D0C5
:1015300022D022D022D022D022D022D022D022D01B
:1015400022D022D022D022D022D022D022D050D0DD
:1015500066D075D08AD094D09ED0ABD0B4D0C6D04F
:1015600019D019D019D0010C000C000C000C000C83
:10157000000C000C000C000C000C000C000C000C0B
:10158000000C000C000C000C000C000C000C000CFB
:10159000000C000C000C000C000C200C000C7C510A
:1015A0000F09706F7D51F00970177039945D01E675
:1015B00003D0030EC9EC03F07E510F09706F7F5109
:1015C000F00970177039955D01E603D0040EC9EC7F
:1015D00003F00D0E756F77512B5C5F08D8B0E10CEE
:1015E000756B1B941B921B801B961B88000C000CB8
:1015F0001BB206D01B82080E726F220E786F4BD082
:1016000090439051909F1D1902E78C0E901B724FD2
:1016100002D01D4340D01B927951756F6DD71BB21C
:1016200005D01B82090E726F230E786F724F03D0A4
:101630006A3326E21AD01B927A51756F5DD71C6A05
:10164000F90ED76EEA0ED66EFF0E676F2A0E666F22
:10165000FB0E696F040E686F8B9EF29E949ED58E72
:10166000F28E1B9078C075F0000C030E1C6EFF0EFE
:10167000D76E4A0ED66EFF0E676FE60E666FECD71A
:10168000030E1C6EFF0ED76EF20ED66EFF0E676F46
:101690003D0E666FE1D71C6AFF0ED76EF20ED66E56
:1016A000FF0E676FE90E666FFF0E696F590E686F68
:1016B000D3D7290E756F1D6ACC0E6A6F290E7A6F0B
:1016C000230E786FBCD71DC071F01DAE08D01B94DF
:1016D000756B1B80A50E876F5A0E866F000C440E2B
:1016E0006A6F2A0E7A6F2BC077F099D71D6A6BC08C
:1016F0006AF07BC07AF0230E786FA1D71BB40FD0AD
:101700001B84BC0EF66E280EF76EF86AA68E0900D2
:10171000F5CF73F0F6CF3CF1F7CF3DF10FD03CC1E0
:10172000F6FF3DC1F7FFF86A080E746F00EE86F011
:10173000A68E0900F5CFEEFF742FFBD7F6CF3CF154
:06174000F7CF3DF112009D
:0A17460080EF02F0020131B600D17D
:1017500031B204D031B406D031901200000E466F81
:10176000318600D1050E466F3186FCD0C00E476F22
:1017700048693651475F3751485B47C236F248C225
:1017800037F21FAA39D089C1E8FF375D01E203D0E3
:10179000050EC9EC03F0820E510351BFF45E780EC2
:1017A000F3265A0EF4223751F402F4CF4AF2F3CF63
:1017B00049F23651F302F4CF4EF2F3CF47F2F4027E
:1017C000F3504E27F4504923E86A4A233751F30275
:1017D000F3504E25486FF4504923E86A4A23D890C5
:1017E0004A334933D8904A334933D8904A3349333E
:1017F00049C267F24AC268F2462B000C1FAC07D000
:1018000039C2E8FFE830E89E800FE8CF78F1462B38
:10181000000C8AC1E8FF3B5D01E203D0060EC9EC73
:1018200003F02F0E500350BFF45E550EF326D00E7A
:10183000F4223B51F402F4CF4AF2F3CF49F23A5189
:10184000F302F4CF4EF2F3CF47F2F402F3504E27F7
:10185000F4504923E86A4A233B51F302F3504E25E2
:10186000486FF4504923E86A4A23D8904A334933F1
:10187000D8904A334933D8904A334933D8904A33C1
:101880004933D8904A334933D8904A33493349C20F
:1018900069F24AC26AF2462B000C8BC1E8FF3D5D3B
:1018A00001E203D0070EC9EC03F01E0E4F034FBF39
:1018B000F45EBC0EF326890EF4223D51F402F4CFFF
:1018C0004AF2F3CF49F23C51F302F4CF4EF2F3CF98
:1018D00047F2F402F3504E27F4504923E86A4A23B2
:1018E0003D51F302F3504E25486FF4504923E86A06
:1018F0004A23D8904A334933D8904A33493349C2AE
:1019000065F24AC266F2462B000C66516A03F4CFB8
:101910004AF2F3CF49F265516903F4CF4EF2F3CFA7
:1019200047F26A03F3504E27F4504923E86A4A23EA
:1019300066516903F3504E25486FF4504923E86A15
:101940004A2348C271F249C272F231923196000CB8
:101950004651080807E23190319231943196336A4A
:10196000466B120046517AEC02F000D747D751D7A8
:1019700094D7CBD704D042D071D0A0D0CFD00D0E09
:10198000530353BFF45E800EF326CF0EF4223F5173
:10199000F402F4CF4AF2F3CF49F23E51F302F4CF0E
:1019A0004EF2F3CF47F2F402F3504E27F45049239E
:1019B000E86A4A233F51F302F3504E25486FF45032
:1019C0004923E86A4A23D8904A334933D8904A33A6
:1019D0004933D8904A334933D8904A334933D89061
:1019E0004A334933D8904A334933D8904A3349333C
:1019F00049C26DF24AC26EF2462B000C0D0E540322
:101A000054BFF45E800EF326CF0EF4223751F40259
:101A1000F4CF4AF2F3CF49F23651F302F4CF4EF24B
:101A2000F3CF47F2F402F3504E27F4504923E86A0B
:101A30004A233751F302F3504E25486FF45049239F
:101A4000E86A4A23D890483749374A37010E4A177F
:101A500049C26DF24AC26EF2462B000C0D0E5503C0
:101A600055BFF45E800EF326CF0EF4223F51F402F0
:101A7000F4CF4AF2F3CF49F23E51F302F4CF4EF2E3
:101A8000F3CF47F2F402F3504E27F4504923E86AAB
:101A90004A233F51F302F3504E25486FF450492337
:101AA000E86A4A23D890483749374A37010E4A171F
:101AB00049C26DF24AC26EF2462B000C0D0E56035F
:101AC00056BFF45E800EF326CF0EF4223F51F4028F
:101AD000F4CF4AF2F3CF49F23E51F302F4CF4EF283
:101AE000F3CF47F2F402F3504E27F4504923E86A4B
:101AF0004A233F51F302F3504E25486FF4504923D7
:101B0000E86A4A23D890483749374A37010E4A17BE
:101B100049C26FF24AC270F2462B000C31943196E2
:021B2000000CB7
:0E1B2200170E80EC02F00101A6B21200A6948C
:101B3000A19808B214D0F29CA69EA96AA680A68E8F
:101B4000F28C90C1E8FF0F0BE8CF90F1A8624DD066
:101B5000006B002BD80E026F220E036F0882A69C2A
:101B6000F86A02C1F6FF03C1F7FFA68E0900F5CFA0
:101B7000E9FF0900F5CFEAFFF6CF02F1F7CF03F155
:101B800008BA10D0F29CA69E00C1A9FFA680EF5013
:101B9000A8621FD8A68EF28C002B0F0E00651200D3
:101BA000088A120090C1E8FF0F0B0D0DF3500025BD
:101BB000A96EF29CA69EA680EF50A8620AD8A68EB7
:101BC000F28C002B1C0E0065120008900892089AF7
:101BD0001200A86E032AA684F29E550EA76EAA0EC6
:101BE000A76EA682A694F28E1200EE0EC9EC03F048
:101BF00090C1E8FF0F0BF29CA69EA96AEADFA68EB1
:101C0000F28CA6B2FED70101006BA69CD60EF66E32
:101C1000220EF76EF86AA68E0900F5CFE9FF0900DB
:101C2000F5CFEAFFA69E00C1A9FFA6800000A8503C
:101C3000EF6E002B0F0E0065EED790C1E8FF0F0B83
:101C40000D0DF3500025A96EA68E0900F5CFE9FF12
:101C50000900F5CFEAFFA69EA6800000A850EF6E0F
:0A1C6000002B1C0E0065E9D71200EE
:061C6A00000C000C060E48
:101C700008B6E8280F6E09980A8208B605D01950F0
:101C8000150F106E09980A8408A602D018BA1A6AAD
:101C9000207420B4209020A420921E741EB408D07A
:101CA0000101090E1EBC0C0E1EA601D0080E7A6F93
:101CB000080E1EA6E8287B6F0A0E1EB8E8287C6F67
:101CC00001012D2A020E2D5CD8A400D0090E2D642E
:101CD00012008A7C088C08A6096A08A60A6A020112
:101CE000F29E13C296F014C297F015C298F0136BCF
:101CF000146B156BF28E01010101F29E74C17DF12E
:101D000075C17EF1746B756BF28E7D513C0DF3CF16
:101D100083F1F4CF84F17E513C0DF350842783C1CD
:101D200093F184C194F1010107B01A6A1A2A08B626
:101D300002D00C0E01D0030E1A6404D008761A6A81
:101D4000096A0A6A2D6A252A2E2A3B0E256414D0B8
:101D500008B6096A08B60A6A256A262A3B0E26646E
:101D60000BD0266A272A170E276406D0276A282A4E
:101D7000630E286401D0286A030E0E6E09980A804B
:021D8000000C55
:0E1D8200210E80EC02F092C123F08E5178EC1D
:101D900002F00BEF03F01DEF03F02FEF03F03DEF28
:101DA00003F0D9EF0EF06DEF03F074EF03F016EFD0
:101DB0000FF0208020821FB60BD01E9891BF1E8886
:101DC0009151D8A41F8604E09145E880786F1CD01B
:101DD0001FA20BD01F921FB404D01E8880C178F1BF
:101DE00013D01E9881C178F10FD018B205D01F8E84
:101DF0001E887FC178F108D018B405D01F8E1E98B8
:101E00007FC178F101D0170C6B686A6A6F6A6F8CBA
:101E1000899092801F921E861E8C010E766F6A6AD0
:101E2000EA0E6B168E2B2CC095F1080C1FAE06D057
:101E300018A21FD018A41DD01F9E17D018B203D00F
:101E4000784F782B16D018B403D0784B786911D01E
:101E50001FA20FD01F921FA608D01EA803D078C1C2
:101E600080F103D078C181F100D01F861E961F98A3
:081E7000776BA2EF03F0150CE3
:1022D000130E80EC02F090013B01330152025102D7
:1022E00050024F028C018B018901940095005B0123
:1022F00059016D0F21007F018701880192018A0138
:1023000082014F015101910158015A01800181015F
:1023100041A042A1E045A3A4A5A64BA74D484FA8C4
:10232000504354A9AA58E1ABACE2ADAE62AFB0B134
:1023300061B2B3B4E365B6B7B8B9BABBBCBD6FBEE2
:102340007063BF79E478E5C0C1E6C2C3C4C5C6C73F
:10235000BA24C024D624EC24F9240125CA23E3237B
:1023600024242C2436244B246024692474247F24C0
:102370008A2495249E24A724B024092522253B25C0
:1023800054258225AD25C425EF251A2645265E262F
:1023900077269026A926C226DB2610272727402746
:1023A000592772278B27A927C527E127FF27182838
:1023B0001828182818281828182831284428572899
:1023C0006B287F2898289828982827182D001A1BF2
:1023D0000116141172012C108E012C108D011A336C
:1023E00001000027182D0016481967021647543DB2
:1023F00016131172011965025616541060002C1044
:102400008F012C165A196902412C13710216675755
:10241000164E197C001640197E002C16071A7A01F8
:102420001A7C01000020139301200000003D3D3D77
:102430003D3D3D3D0000001600CFF0FFECEE3E3E7E
:10244000160D3D10780120D1EAF00000160020534F
:1024500070641078013D160E3CCEE1F0E0F2001AF7
:10246000003DD1D2CECF3D3D0000D1E2E5F0F520D8
:10247000D2EEEA0000D1E2E5F0F5CDE0EFF00000A9
:10248000D1E2E5F0F5D2E5ECEF0000CCE0EBEEE5D3
:10249000CDE0EFF000002020202052554E0000201B
:1024A000202052554E200000202052554E20200062
:1024B000002052554E202020000000280C0601006C
:1024C00014537461727420544553542052696768E0
:1024D00074204B65790014436F6E74696E75652DB9
:1024E0004D6964646C65204B657920001F122700DC
:1024F0003A1226003A12250000001600FF1613FFBC
:1025000000001600201613200001121900C7E0F980
:102510002E20C4F0E5E1E5E7E3E03D17031C123BA4
:1025200001000112190020CDEEECE5F020CCEEF216
:10253000EEF0E03D17000F1090010001121900C2EB
:10254000E5F0F5CFEEF0EEE3D2EEEAE03D1701FF65
:10255000108A010001121900202020D3F1EAEEF0C8
:10256000E5EDE8E5203D1701FF109201164053709C
:10257000643D107F012C204D61785370643D1082C2
:10258000010001121900D1EAEEF0EEF1F2FC20CFC9
:10259000EEEBFF3D1701FF107F01164052504D3DFD
:1025A0001393012C20416D703D117201000112192D
:1025B00000C0E2F2EE20D1F2E0F0F23D2017000080
:1025C0001491010001121900CDE0F72E20CCEEE4A9
:1025D000F3EBFFF62E3D1700FF10880116405370F5
:1025E000643D107F012C20416D703D11720100018E
:1025F000121900D3F1E8EB2ECCEEE4F3EBFFF62E4C
:102600003D1700FF10870116405370643D107F0195
:102610002C20416D703D1172010001121900C8EDAE
:10262000E42ECCE0EAF1D1EAEEF02E3D1700FF10E7
:10263000820116405370643D107F012C2052504D92
:102640003D1393010001121900C8EDE42ED7E0F10B
:10265000F22ED8C8CC203D170014124F01000112F1
:102660001900D3E3EEEBCCE5E6E4F3D4E0E7203D5C
:102670001700031251010001121900CFF0EEE3F030
:102680002ED3EFF0E0E2EB2E3D17000A12580100C6
:1026900001121900CDE8E7EAEEE520CDE0EFF0FF0A
:1026A000E63D1700FF108C010001121900C2FBF17A
:1026B000EEEAEEE5CDE0EFF0FFE63D1700FF108B10
:1026C000010001121900D2E5F0ECE8F1F2EEF02081
:1026D000C7E0F93D1700FF108901000112190057EA
:1026E0003120D2E5ECEF2EC7E0F93D17837D14943D
:1026F0000016401086001087001088001089001016
:102700008A00108B00108C00108D002C109000009F
:1027100001121900573120C7E0F9E8F2E020313DFD
:1027200017837D1495000001121900CAEEECEFE545
:10273000EDF1E0F6E8FF44433D1700FF105A0100B9
:1027400001121900CDEEECE8EDE0EBFCEDEEE54416
:10275000433D1700FF105B010001121900C2F0E5B4
:10276000ECFFC7E0F0FFE4CAEDE43D1700FF1059AD
:10277000010001121900C8EDF2E5F0E2E0EB44546B
:10278000434F4E3D17003F106D0F0001121900CD51
:10279000EEEBFC20E8E7EC2EF2EEEAE03D1700005D
:1027A0001052021640113A020001121900D0E5E35E
:1027B000F3EBFC20D2EEEAE03D17000014500216C5
:1027C00040113A020001121900CDE0EFF020EFEEC7
:1027D000E4F1F2F03D170000144F021640113C02E4
:1027E0000001121900D2E5F0ECE8F1F22ECAEEF089
:1027F0003D1700001451021640543D1967020001B4
:10280000121900C2E0F0E8E0EDF2203420F1F2F01D
:102810003D17353A1233010001121900C7E0E4E513
:10282000F0E6EAE020D2E5F1F23D1701FF102100C9
:1028300000541654313D196502562C196902412C79
:1028400010180000541654323D196702432C196BBE
:1028500002412C10170000541654333D19690256DA
:102860002C196D0241002C00000000541654343D18
:10287000196B02562C196F0241002C000000005405
:1028800016541136024D3D111C0220204510320015
:102890001022002010170000541654353D10370246
:1028A000103902103B02103D02103F02104102108D
:1028B0004302104502202000000000000328475179
:1028C000EE09000064285920ED09000004284C702E
:1028D000390100000BD20F483F004F050E1438009D
:1028E00046380CE030003D9F0A7C2A00353809E06C
:1028F00024002E0508142000280507141C002305B9
:10290000061418001E3805E014001A9F047C1200FB
:10291000170504141000146B03AC0D00110503140B
:102920000C000F9F027C0A000D3802E008000B0526
:10293000021408000AD201480700099F017C060022
:10294000086B01AC0500073801E00400060501141E
:10295000040005333333FFFF7FFFFF3FFFFF7FCCD2
:10296000CC4CFFFF7F555555AAAAAAE107E107E124
:1029700007E107E107E107E107E107E007E007E01A
:1029800007E007E007DF07DF07DF07DF07DE07DE17
:1029900007DE07DD07DD07DC07DC07DC07DB07DB1D
:1029A00007DA07DA07D907D807D807D707D707D62E
:1029B00007D507D507D407D307D307D207D107D048
:1029C00007CF07CF07CE07CD07CC07CB07CA07C96C
:1029D00007C807C707C607C507C407C307C207C19B
:1029E00007C007BF07BE07BD07BB07BA07B907B8CF
:1029F00007B707B507B407B307B107B007AF07AD0F
:102A000007AC07AA07A907A807A607A507A307A257
:102A100007A0079E079D079B079A079807960795AB
:102A200007930791078F078E078C078A0788078708
:102A3000078507830781077F077D077B077907776E
:102A4000077507730771076F076D076B07690767DE
:102A5000076507630760075E075C075A0758075555
:102A600007530751074E074C074A074707450743D7
:102A70000740073E073B0739073607340731072F62
:102A8000072C072A072707250722071F071D071AF4
:102A9000071707150712070F070C070A0707070490
:102AA000070107FE06FC06F906F606F306F006ED3A
:102AB00006EA06E706E406E106DE06DB06D806D5EA
:102AC00006D206CF06CC06C806C506C206BF06BC9F
:102AD00006B806B506B206AF06AB06A806A506A15F
:102AE000069E069B069706940691068D068A068624
:102AF0000683067F067C067806750671066D066AF3
:102B000006660663065F065B065806540650064DC9
:102B1000064906450641063E063A06360632062EA8
:102B2000062B06270623061F061B06170613060F8D
:102B3000060B0607060306FF05FB05F705F305EF81
:102B400005EB05E705E305DF05DB05D605D205CE78
:102B500005CA05C605C205BD05B905B505B105AC73
:102B600005A805A4059F059B05970592058E058977
:102B700005850581057C05780573056F056A056681
:102B80000561055D05580554054F054B0546054192
:102B9000053D05380533052F052A05250521051CAA
:102BA00005170513050E05090504050005FB04F6C8
:102BB00004F104EC04E804E304DE04D904D404CFF3
:102BC00004CA04C504C004BB04B604B204AD04A81E
:102BD00004A3049E04990494048E04890484047F4D
:102BE000047A04750470046B04660461045B045683
:102BF0000451044C04470442043C04370432042DBD
:102C000004270422041D04180412040D04080402FD
:102C100004FD03F803F203ED03E803E203DD03D749
:102C200003D203CD03C703C203BC03B703B103AC94
:102C300003A603A1039B03960390038B03850380E4
:102C4000037A0375036F036A0364035E0359035336
:102C5000034E03480342033D03370331032C03268D
:102C60000320031B0315030F030A030403FE02F8EA
:102C700002F302ED02E702E102DC02D602D002CA50
:102C800002C502BF02B902B302AD02A802A2029CB1
:102C900002960290028A0284027F02790273026D18
:102CA00002670261025B0255024F024A0244023E81
:102CB00002380232022C02260220021A0214020EEC
:102CC0000208020202FC01F601F001EA01E401DE61
:102CD00001D801D201CC01C601C001BA01B401AED4
:102CE00001A801A2019C0196019001890183017D47
:102CF00001770171016B0165015F01590153014DBC
:102D000001470140013A0134012E01280122011C32
:102D10000116010F0109010301FD00F700F100EBAD
:102D200000E400DE00D800D200CC00C600C000B92C
:102D300000B300AD00A700A1009B0094008E0088A6
:102D40000082007C0076006F00690063005D005720
:102D50000050004A0044003E00380031002B00259E
:102D6000001F00190013000C0006000000FAFFF419
:102D7000FFEDFFE7FFE1FFDBFFD5FFCFFFC8FFC29D
:102D8000FFBCFFB6FFB0FFA9FFA3FF9DFF97FF9118
:102D9000FF8AFF84FF7EFF78FF72FF6CFF65FF5F95
:102DA000FF59FF53FF4DFF47FF40FF3AFF34FF2E0F
:102DB000FF28FF22FF1CFF15FF0FFF09FF03FFFD88
:102DC000FEF7FEF1FEEAFEE4FEDEFED8FED2FECC09
:102DD000FEC6FEC0FEB9FEB3FEADFEA7FEA1FE9B81
:102DE000FE95FE8FFE89FE83FE7DFE77FE70FE6AF5
:102DF000FE64FE5EFE58FE52FE4CFE46FE40FE3A6B
:102E0000FE34FE2EFE28FE22FE1CFE16FE10FE0ADA
:102E1000FE04FEFEFDF8FDF2FDECFDE6FDE0FDDA50
:102E2000FDD4FDCEFDC8FDC2FDBCFDB6FDB1FDABC0
:102E3000FDA5FD9FFD99FD93FD8DFD87FD81FD7C29
:102E4000FD76FD70FD6AFD64FD5EFD58FD53FD4D90
:102E5000FD47FD41FD3BFD36FD30FD2AFD24FD1FF4
:102E6000FD19FD13FD0DFD08FD02FDFCFCF6FCF156
:102E7000FCEBFCE5FCE0FCDAFCD4FCCFFCC9FCC3B9
:102E8000FCBEFCB8FCB2FCADFCA7FCA2FC9CFC9612
:102E9000FC91FC8BFC86FC80FC7BFC75FC70FC6A66
:102EA000FC65FC5FFC5AFC54FC4FFC49FC44FC3EB6
:102EB000FC39FC33FC2EFC29FC23FC1EFC18FC1303
:102EC000FC0EFC08FC03FCFEFBF8FBF3FBEEFBE84E
:102ED000FBE3FBDEFBD9FBD3FBCEFBC9FBC4FBBE94
:102EE000FBB9FBB4FBAFFBAAFBA5FB9FFB9AFB95D1
:102EF000FB90FB8BFB86FB81FB7CFB77FB72FB6C07
:102F0000FB67FB62FB5DFB58FB53FB4EFB4AFB453B
:102F1000FB40FB3BFB36FB31FB2CFB27FB22FB1D65
:102F2000FB18FB14FB0FFB0AFB05FB00FBFCFAF78D
:102F3000FAF2FAEDFAE9FAE4FADFFADBFAD6FAD1B4
:102F4000FACDFAC8FAC3FABFFABAFAB5FAB1FAACCE
:102F5000FAA8FAA3FA9FFA9AFA96FA91FA8DFA88E1
:102F6000FA84FA7FFA7BFA77FA72FA6EFA69FA65EE
:102F7000FA61FA5CFA58FA54FA4FFA4BFA47FA43F4
:102F8000FA3EFA3AFA36FA32FA2EFA2AFA25FA21F3
:102F9000FA1DFA19FA15FA11FA0DFA09FA05FA01E9
:102FA000FAFDF9F9F9F5F9F1F9EDF9E9F9E5F9E1E0
:102FB000F9DDF9D9F9D5F9D2F9CEF9CAF9C6F9C2CC
:102FC000F9BFF9BBF9B7F9B3F9B0F9ACF9A8F9A5AC
:102FD000F9A1F99DF99AF996F993F98FF98BF98886
:102FE000F984F981F97DF97AF976F973F96FF96C59
:102FF000F969F965F962F95FF95BF958F955F95121
:10300000F94EF94BF948F944F941F93EF93BF938E1
:10301000F934F931F92EF92BF928F925F922F91F9C
:10302000F91CF919F916F913F910F90DF90AF9074C
:10303000F904F902F9FFF8FCF8F9F8F6F8F4F8F1F8
:10304000F8EEF8EBF8E9F8E6F8E3F8E1F8DEF8DB9B
:10305000F8D9F8D6F8D4F8D1F8CFF8CCF8CAF8C730
:10306000F8C5F8C2F8C0F8BDF8BBF8B9F8B6F8B4BE
:10307000F8B2F8AFF8ADF8ABF8A8F8A6F8A4F8A243
:10308000F8A0F89DF89BF899F897F895F893F891BF
:10309000F88FF88DF88BF889F887F885F883F88130
:1030A000F87FF87DF87BF879F878F876F874F8729C
:1030B000F871F86FF86DF86BF86AF868F866F865FB
:1030C000F863F862F860F85EF85DF85BF85AF85853
:1030D000F857F856F854F853F851F850F84FF84D9F
:1030E000F84CF84BF849F848F847F846F845F843E3
:1030F000F842F841F840F83FF83EF83DF83CF83B1C
:10310000F83AF839F838F837F836F835F834F8334B
:10311000F832F831F831F830F82FF82EF82DF82D74
:10312000F82CF82BF82BF82AF829F829F828F82891
:10313000F827F826F826F825F825F824F824F824A6
:10314000F823F823F822F822F822F821F821F821B0
:10315000F821F820F820F820F820F820F81FF81FB0
:10316000F81FF81FF81FF81FF81FF81FF81FF81FA7
:10317000F81FF81FF81FF81FF81FF8010003002FB1
:10318000003B00490059006700710089009500A3C9
:1031900000B300C100D300DF00EF00FB000D011BF6
:1031A00001250139014B015B016701750185019121
:1031B00001A301AF01BB01CD01DF01EB01F7010963
:1031C000021D0223023302410251025F026B02819F
:1031D000028D02A102AB02BD02C502D702E702F5D1
:1031E00002050313031D0335033D0355035F036D00
:1031F0000377038B039703A903B903C703D703E539
:1032000003F103FD030F041B042D043F0449045D77
:103210000469047F048B049304A304B104C104CFA4
:1032200004E104EB04FD040B051B0529052F0551E2
:1032300005570565057705810593059F05AD05BF14
:1032400005CF05DB05E705FB050706170623062F57
:103250000647065306650679067F0685069D06AD78
:1032600006BB06CD06D906DF06F706090713071FBA
:1032700007370745074F0761076D0779078B079DDC
:10328000079F07B507C907D307E107F70705080F29
:1032900008210833083F0851085908690871088354
:1032A000089B08A508AD08C308CB08E108EF08F99A
:1032B0000807091D092B093509490959096B0977BF
:1032C0000985098F09A309AD09C709C709D909EB00
:1032D00009FD09130A130A210A390A490A570A6320
:1032E0000A6F0A810A930A9F0AAB0ABD0ACF0AD95C
:1032F0000AE70AF30A030B150B230B2D0B3F0B51A7
:103300000B5D0B6F0B7B0B8D0B9B0BB70BB90BC3C3
:103310000BCF0BE10BF50B070C110C250C2F0C41FF
:103320000C410C5B0C6D0C770C890C950C9D0CB54D
:103330000CC70CC70CE30CF10C010D0F0D1F0D2B6E
:103340000D3D0D4F0D550D690D790D850D8D0DA39D
:103350000DAB0DBD0DCD0DDB0DE70DFD0D090E17F0
:103360000E270E350E4B0E570E5D0E710E7D0E8F15
:103370000E9B0EB10EB90ED10EDB0E5D0100BD022B
:1033800000190400770500D306003308008F0900F8
:10339000ED0A00410C00AB0D00070F00691000C3DF
:1033A0001100191300751400D715003317008F187A
:1033B00000ED19004F1B00A51C000B1E00671F002D
:1033C000C52000212200832300DD24003B26009B32
:1033D0002700F72800552A00A92B00072D006F2E83
:1033E00000CF2F002731008D3200EB330041350034
:1033F0008F3600F737005B3900B73A00113C007395
:103400003D00C93E002B4000934100E3420045448B
:1034100000A345000547005B4800B54900134B0079
:10342000734C00D74D002D4F00935000F551004BC9
:103430005300A954000B5600615700C158001F5A91
:1034400000795B00D75C00395E00955F00F5600095
:10345000516200B363000B6500616600C16700291B
:1034600069007B6A00DB6B00396D00956E00F56FBB
:1034700000517100B372001574006B7500C37600C3
:10348000257800917900ED7A00377C009F7D00FB64
:103490007E004B8000B381000B8300778400CD85D4
:1034A000002B8700858800EF8900578B009F8C00D8
:1034B000018E00598F00B99000159200739300E1BE
:1034C0009400319600939700E398004B9A00A79BD5
:1034D00000019D005F9E00C19F001BA10079A2001A
:1034E000D5A30035A50093A600EDA70043A900AB26
:1034F000AA0009AC0065AD00C5AE001BB0007FB1ED
:1035000000D3B2003DB40099B500EFB60055B80045
:10351000ADB90009BB006FBC00CDBD0033BF007F5B
:10352000C000E1C10047C3009DC400FBC50057C7F0
:1035300000B7C80009CA0071CB00D1CC002FCE0063
:1035400089CF00E7D00047D200A5D300F9D4005DB1
:10355000D600BDD7001BD90077DA00CDDB0035DD02
:103560000097DE00F1DF0043E100ABE20001E40080
:1035700067E500BDE6001BE8007BE900DFEA002903
:10358000EC0095ED00F1EE004FF000AFF1000BF311
:103590000063F400C9F5002DF70081F800E9F90097
:1035A0003FFB0097FC00F3FD004DFF00B10001134D
:1035B00002016D0301CB04011F06017D0701DF0835
:1035C00001410A019B0B01FF0C01530E01B50F01D4
:1035D000171101691201CF13012D15017D1601DFAD
:1035E00017013F1901A11A01FD1B01531D01AB1E5B
:1035F00001172001732101D122012D24018D250104
:10360000EF26014D2801AF2901FF2A016B2C01BBD8
:103610002D01172F017F3001DD31013333018D344E
:1036200001E935014D3701A73801033A01613B013A
:10363000C93C011F3E01873F01DB40013742019534
:103640004301E94401514601B347010F49016D4A65
:1036500001D34B01314D01874E01E74F0145510127
:10366000955201FD5301575501BB56010F58016B8F
:103670005901C35A01235C01855D01BD0200770534
:1036800000330800ED0A00AB0D00691000191300AB
:10369000D715008F18004F1B000B1E00C52000839C
:1036A00023003B2600F72800A92B006F2E002731AE
:1036B00000EB33008F36005B3900113C00C93E003F
:1036C000934100454400054700B54900734C002D67
:1036D0004F00F55100A954006157001F5A00D75CF4
:1036E00000955F005162000B6500C167007B6A00B6
:1036F000396D00F56F00B372006B7500257800ED31
:103700007A009F7D004B80000B8300CD850085886B
:1037100000578B00018E00B9900073930031960022
:10372000E39800A79B005F9E001BA100D5A3009318
:10373000A60043A90009AC00C5AE007FB1003DB4AE
:1037400000EFB600ADB9006FBC0033BF00E1C100AF
:103750009DC40057C70009CA00D1CC0089CF0047DB
:10376000D200F9D400BDD70077DA0035DD00F1DFF3
:1037700000ABE20067E5001BE800DFEA0095ED0022
:103780004FF0000BF300C9F50081F8003FFB00F398
:10379000FD00B100016D03011F0601DF08019B0B55
:1037A00001530E01171101CF13017D16013F1901BD
:1037B000FD1B01AB1E017321012D2401EF2601AF7A
:1037C00029016B2C01172F01DD31018D34014D379B
:1037D00001033A01C93C01873F01374201E9440135
:1037E000B347016D4A01314D01E74F019552015731
:1037F00055010F5801C35A01855D013D6001076302
:1038000001B965016D68013B6B01F36D01AB70019E
:103810005F73011D7601D57801917B014F7E010315
:103820008101BB83017986013D8901F38B01AD8E56
:1038300001699101219401E19601939901559C013F
:10384000159F01CDA1017FA40147A701F9A901B7E7
:10385000AC017BAF012DB201E7B4019FB70151BAB2
:10386000011BBD01D3BF018FC20149C50105C801BC
:10387000C3CA0183CD013BD001EDD201A9D50169B5
:10388000D80125DB01D7DD0197E00155E30111E601
:1038900001CBE8017DEB0135EE01F3F001BBF30153
:1038A00075F60121F901E5FB01A9FE01670102118D
:1038B0000402D106028F09024B0C02050F02C1114E
:1038C000027F1402451702F11902A71C02651F02AC
:1038D000252202E92402992702532A020F2D02BB56
:1038E0002F027F32023D3502F73702B33A02713DB3
:1038F000022F4002E742029B45026348021B4B0233
:10390000CF4D028D5002495302015602D958027D13
:103910005B02375E02EF6002AD63026B66022769ED
:1039200002EB6B029D6E025171020D7402BF7602B2
:10393000A17902417C02F57E02B781027B840229D3
:103940008702DB89029F8C025B8F020F9202D9945F
:1039500002839702539A02079D02AB9F0277A2024D
:103960002FA502F3A702ABAA0267AD0221B002D9CC
:10397000B20291B50253B80207BB02770500ED0A07
:1039800000691000D715004F1B00C520003B260022
:10399000A92B002731008F3600113C009341000510
:1039A0004700734C00F55100615700D75C0051622D
:1039B00000C16700396D00B372002578009F7D005B
:1039C0000B8300858800018E00739300E398005FED
:1039D0009E00D5A30043A900C5AE003DB400ADB91B
:1039E0000033BF009DC40009CA0089CF00F9D4008C
:1039F00077DA00F1DF0067E500DFEA004FF000C989
:103A0000F5003FFB00B100011F06019B0B011711E0
:103A1000017D1601FD1B01732101EF26016B2C01B5
:103A2000DD31014D3701C93C01374201B347013156
:103A30004D019552010F5801855D010763016D68C5
:103A400001F36D015F7301D578014F7E01BB8301E6
:103A50003D8901AD8E01219401939901159F017F4C
:103A6000A401F9A9017BAF01E7B40151BA01D3BFA9
:103A70000149C501C3CA013BD001A9D50125DB011C
:103A800097E00111E6017DEB01F3F00175F601E528
:103A9000FB01670102D106024B0C02C1110245175E
:103AA00002A71C022522029927020F2D027F320253
:103AB000F73702713D02E74202634802CF4D0249E7
:103AC0005302D95802375E02AD63022769029D6E28
:103AD000020D7402A17902F57E027B8402DB890269
:103AE0005B8F02D99402539A02AB9F022FA502ABBF
:103AF000AA0221B00291B50207BB0289C002F7C534
:103B0000026FCB02E9D0025BD602D5DB0251E102A3
:103B1000C3E60231EC02A3F10213F70295FC021195
:103B20000203810703FB0C03711203E91703651DF0
:103B300003CF2203452803BF2D03353303B93803D0
:103B40001B3E039F43030D49037F4E03FB53036F4B
:103B50005903E55E03556403D16903416F03B774EC
:103B600003357A03A37F031B8503918A0311900316
:103B70008D9503FF9A0369A003E9A50359AB03D10F
:103B8000B0033FB603BDBB0339C103A7C6031DCCB9
:103B90000393D1030FD70387DC03FDE1036BE70336
:103BA000E1EC0363F203CFF7034BFD03C502041DF1
:103BB0000804950D041D13049718041B1E047F238D
:103BC00004ED2804712E04DF3304573904CB3E047E
:103BD000434404BF49042D4F04A95404255A0495B5
:103BE0005F04076504896A04F36F047F7504E37A50
:103BF00004558004B98504458B04BD9004319604B6
:103C0000A79B041DA10495A6040FAC047FB104FD7D
:103C1000B6046BBC04EFC1044BC704C9CC043FD24B
:103C200004BBD7043DDD0499E20421E80493ED04CC
:103C300009F30479F804FBFD045F0305DF0805556B
:103C40000E05CD13054D1905B31E05212405A52923
:103C500005252F05953405FF39057D3F05F1440500
:103C6000614A05F54F05595505DD5A05476005AF11
:103C70006505276B059D7005197605ED0A00D715BA
:103C800000C52000A92B008F3600934100734C0023
:103C9000615700516200396D002578000B830001E7
:103CA0008E00E39800D5A300C5AE00ADB9009DC459
:103CB0000089CF0077DA0067E5004FF0003FFB0096
:103CC0001F0601171101FD1B01EF2601DD3101C99E
:103CD0003C01B34701955201855D016D68015F7339
:103CE000014F7E013D8901219401159F01F9A90130
:103CF000E7B401D3BF01C3CA01A9D50197E0017D93
:103D0000EB0175F6016701024B0C024517022522F3
:103D1000020F2D02F73702E74202CF4D02D95802B7
:103D2000AD63029D6E02A179027B84025B8F025318
:103D30009A022FA50221B00207BB02F7C502E9D003
:103D400002D5DB02C3E602A3F10295FC0281070360
:103D5000711203651D034528033533031B3E030D14
:103D60004903FB5303E55E03D16903B77403A37FE3
:103D700003918A038D950369A00359AB033FB603F2
:103D800039C1031DCC030FD703FDE103E1EC03CFE1
:103D9000F703C50204950D049718047F2304712EC0
:103DA000045739044344042D4F04255A040765047D
:103DB000F36F04E37A04B98504BD9004A79B0495CE
:103DC000A6047FB1046BBC044BC7043FD2043DDDA5
:103DD0000421E80409F304FBFD04DF0805CD130505
:103DE000B31E05A529059534057D3F05614A055992
:103DF0005505476005276B051976052D8105E98B6B
:103E000005E39605C9A105B9AC059FB70593C205A1
:103E10007FCD0569D80555E30541EE051DF9051F60
:103E20000406070F06ED1906C72406BF2F06BB3A86
:103E300006A14506995006755B066566065771062C
:103E4000437C062587060B92060D9D06F9A706DF23
:103E5000B206C7BD06ADC806A9D30691DE0677E94E
:103E60000667F4064DFF06450A072B15070D2007C8
:103E7000FD2A07EF3507D74007CD4B07AD5607A7FB
:103E800061078B6C077977075182074F8D0741983F
:103E90000727A30715AE0701B907EDC307D7CE075C
:103EA000C3D907B7E407A7EF0787FA076D050867C7
:103EB0001008511B083D26082531080F3C08FD4617
:103EC00008E95108DB5C08CB6708B17208997D08E6
:103ED0008B88087B93085B9E084FA90835B4083F80
:103EE000BF0813CA0803D508F1DF08DBEA08C1F5EB
:103EF00008AD0009990B097B1609732109632C0988
:103F0000553709474209234D09135809F96209EB4E
:103F10006D09D77809CB8309AB8E0997990981A4DC
:103F20000975AF095BBA094DC50939D00931DB09FB
:103F30000FE609FDF009E3FB09D9060ABB110AA542
:103F40001C0A9D270A8F320A6F3D0A63480A4753AD
:103F50000A3F5E0A25690A11740AE77E0AE5890AA2
:103F6000BD940ABD9F0AADAA0A8DB50A87C00A6D25
:0B3F7000CB0A4DD60A4FE10A2FEC0AE5
:020000040030CA
:01000100C539
:010002000BF2
:0100030020DC
:0100040024D7
:010005001DDD
:010006008178
:0200000400F00A
:100000000E05350645080901D44870658A0A0C01B9
:1000100007BB462778000A03750110203001010153
:10002000F1510005031100010101020202F2520028
:1000300005030200020202030303F3530005030356
:1000400000030303040404F4540004030400040440
:1000500004050505F555000503050005050506061B
:1000600006F6560006030600060606070707F757BA
:100070000007030700070707080808F858000803E7
:100080000800080808090909F959000903090009C5
:100090000909101010E060000A0310001010101180
:1000A0001111E161000B031100111111121212E282
:1000B00062000C031200121212131313E363000DFB
:1000C000031300131313639D35FF2A24090304014E
:1000D00014281401EEE63399040A0177039988661F
:00000001FF
